:020000040000FA
:040000008A11052834
:100008000900FC21A82183160313071705140612FB
:100018008612013083120313DA00D9011122E0019C
:10002800DF01EC30D200F430D3001E30DB00DC01FD
:100038000F30DD000130B000D401D501D601D70161
:10004800B9010130BA00831203178D018F018312A1
:100058000313AB25831203170C0883120313BC0088
:100068000A30F200F3018A213C08163C031CBC014B
:10007800C220F430F2000130F3008A215D20013003
:10008800C100AB01AC01D401D501AF014103031D8F
:100098004F2827245A2802304102031D5528D02012
:1000A8005A2803304102031D5A28E1224A286300D6
:1000B8005B28B00803198B28B6010230B5007F22EF
:1000C8003030F2000130F300F830F7000530F80066
:1000D800BE253030C5000130C600C222E830F2002B
:1000E8000330F3008A21C220B001B6010130B50007
:1000F8007F223030F2000130F300FE30F700053087
:10010800F800BE253030C5000130C600C222B60155
:100118000630B5007F223C08DE0097222730C50054
:100128000130C600C22A051CC1280A30F200F301BA
:100138008A21A201051CA6280A30F200F3018A21AF
:10014800A20A9E282208283C0318C028BC0A3C089A
:10015800163C031CBC01831203178D018F01831207
:1001680003133C08831203178C008312031398218E
:100178000A30F200F3018A215D200800871201305D
:10018800B40036220430F200F3018A218030B40032
:1001980036220C30F5008229E030F2000430F300FA
:1001A8008A21B101B10ADC30F2000530F3008A215E
:1001B8001930BD00042645303107840083175808DC
:1001C800800028303102031CD6280330C100080003
:1001D800A301A401A501A601A701A801A901AA01DB
:1001E800B301B201B20AB30A101052088E005308C4
:1001F8008F000C1010140830A000EF233F08C00037
:100208003303031D0E294008A30700300318013EDD
:10021800A4072E2902303302031D19294008A50717
:1002280000300318013EA6072E2903303302031DB0
:1002380024294008A70700300318013EA8072E29E3
:1002480004303302031D2E294008A9070030031883
:10025800013EAA073308033C031CB3010C1C3229D6
:100268001C303202031CF6282308F9002408FA007F
:100278002708F5002808F6003725701C4A292708A2
:10028800A3022808031C013EA402522923082702BE
:10029800A3002408031C013E2802A4002508F90035
:1002A8002608FA002908F5002A08F6003725701CE8
:1002B80064292908A5022A08031C013EA6026C2904
:1002C80025082902A5002608031C013E2A02A600CB
:1002D8002508A30726080318013EA4072308F900E8
:1002E8002408FA005B08F5005C08F6003725701C46
:1002F80080290130AD008129AD0108000530F000EA
:10030800F00B84290000F50B82290800F30A043059
:10031800F100A530F000F00B8F29F10B8D29F20BBD
:100328008B29F30B8B290800831603178C130C15E4
:1003380055308D00AA308D008C140C118C18A22910
:100348000C11831203130800831603138712071274
:100358000A30F200F301831203138A217722B708C7
:100368000319B22987128316031307108710071180
:1003780087110F30F200F301831203138A21071447
:10038800871407118711C829C9290716CB29CC2931
:1003980007120530F200F3018A210330C90007165D
:1003A800D529D62907128530F000F00BD929C90BB9
:1003B800D3290530F200F3018A21071087140711A9
:1003C8008711E629E7290716E929EA2907122130C2
:1003D800F000F00BED292830B40036220630B400C6
:1003E80036220C30B4003622C2200C30B800080087
:1003F80000007030831603138F04831203139F13B6
:100408001F10831203179E019F019A1399138312D9
:1004180003138501860187010800D9080319202ADA
:10042800103059020319202A203059020319202AB2
:1004380030305902031DD901101859145A03031DED
:10044800272AD910D91102305A02031D2D2AD9148E
:10045800D91103305A02031D332AD914D915590862
:1004680090000800831603130710871007118711DF
:10047800831203130710871007118711B41B871500
:10048800341B0715B41A8714341A07144B2A071695
:100498004D2A4E2A0712502A512A07108710071191
:1004A8008711B419871534190715B4188714341827
:1004B80007145E2A0716602A612A0712632A642A2B
:1004C80087110711871007103530F000F00B6A2AE2
:1004D800103034020318762A3408073C0318762AA9
:1004E8003408B80008000A30F200F3018A21FF300E
:1004F800B7000800080087123608013C0318882A4C
:100508000230B6021430B5073608F5004030F9005D
:10051800B22535087007CB0080304B04B400362272
:100528000530F50082290A305E020318B42A5E08F5
:10053800D000D1018D242730F2000130F300F601FC
:100548000230F7000630F800C8252A30F7000130DD
:10055800F800552527308400831776088000C12AC3
:100568005E08D000D1018D242730F2000130F3005D
:100578002A30F7000130F8004625080045088400B5
:100588008313461883170008BE00BE080319080025
:100598008716C70101303E02031CE02AC70A470834
:1005A800450784008313461883170008B4003622D1
:1005B8003E084702031CD22A0800B201B20A45309D
:1005C80032078400831700085D020318F22A4530B9
:1005D80032078400831701308000F72A453032073C
:1005E80084008317800128303202031CE22A831218
:1005F80003174A08013C83120313CB008312031725
:100608005408013C83120313CD0060085F05CE0037
:100618004B05CF004D05CB004B1C342B0130AE00F1
:10062800B601B5017F223030F2000130F300E1302D
:10063800F7000530F800BE253030C5000130C6008F
:10064800C222B6010630B5007F223C08DE009722A0
:100658002730C5000130C600C22286160612B9012D
:10066800831203174A08013C83120313CB00831239
:100678000317540583120313CD004D1C5D2BAE01E7
:10068800AF01B601B5017F223030F2000130F3002E
:10069800E930F7000530F800BE253030C5000130DC
:1006A800C600C2223908013CCB004B1C5D2B8612C8
:1006B80006162F08013CCB002E084B05CD004D1C1B
:1006C8007D2BBC0A3C08163C031CBC018312031793
:1006D8008D018F01831203133C08831203178C00CA
:1006E8008312031398210A30F200F3018A210130A2
:1006F800AF005F08013CCB0060084B05CD008312BA
:1007080003174A0583120313CB00831203175405FA
:1007180083120313CD004D1C932B0130B9008312B3
:1007280003175408013C83120313CB0083120317E9
:100738004A08831203134B05CD004D1CB62B01301C
:10074800B900B601B5017F223030F2000130F30064
:10075800F130F7000530F800BE253030C500013013
:10076800C600C2225F08013CCB00831203174A0867
:10077800013C83120313CD0060084B05CE004D05E4
:10078800CB0083120317540583120313CD004D1CAD
:10079800E02B0130B900B601B5017F223030F200FC
:1007A8000130F300F130F7000530F800BE25303095
:1007B800C5000130C600C222831203174A088312FB
:1007C8000313E00083120317540883120313DF0096
:1007D8000130C10008009F13831203179E019F0177
:1007E80083120313200AA1000314831203179E0D1A
:1007F8009F0D83120313A10BF92B831603131F13E9
:100808009F161F16831203131F119F111F129F1289
:1008180020181F15A0189F1520191F16A0199F161C
:100828001F140230F50082219F1400009F181A2C13
:100838001F10831203179E019F01831203131E08C2
:10084800BF009F130800EC202D03031D402CBA01A4
:100858002E03031D302C06121830BD000426580A3A
:10086800BB000130C1003B085D020318402C3B0867
:10087800C2000230C1000800B9080319652C013014
:10088800F200F3018A21D40A0319D50A5408F500A5
:100898005508F6000730F900FA013725701C572C67
:1008A80086160612592C861206165408F9005508A1
:1008B800FA000D30F500F6013725701C652CD401BF
:1008C800D501BA0803198A2C0130F200F3018A21F4
:1008D800D60A0319D70A5608F5005708F6000D304E
:1008E800F900FA013725701C7C2C861206127E2C22
:1008F800861206165608F9005708FA001A30F5004D
:10090800F6013725701C8A2CD601D7019720272C91
:100918000800C4015008F5005108F6001030F9002D
:100928002730FA003725F009701CB22C5008F50062
:100938005108F6001030F9002730FA0073257508C1
:10094800CA007008D0007108D100C40A2A304407D0
:100958008400831730304A078000BE2C5008F50009
:100968005108F600E830F9000330FA003725F0099D
:10097800701CD62C5008F5005108F600E830F90034
:100988000330FA0073257508CA007008D000710892
:10099800D100C40A2A3044078400831730304A073C
:1009A8008000E12C5008F5005108F6006430F90089
:1009B800FA013725F009701CF82C5008F500510889
:1009C800F6006430F900FA0173257508CA0070084A
:1009D800D0007108D100C40A2A3044078400831764
:1009E80030304A078000032D5008F5005108F60002
:1009F8000A30F900FA013725F009701C192D500842
:100A0800F5005108F6000A30F900FA017325750857
:100A1800CA007008D0007108D100C40A2A304407FF
:100A28008400831730304A078000C40A2A304407FC
:100A3800840083173030500780007008D000710898
:100A4800D100440883120317AA0083120313080075
:100A5800F00175087902031D080076087A02031D63
:100A68000800F0090800F00176087A02031C080063
:100A78007A087602031C442D7908750203180800C9
:100A8800F009080077088400831378188317000892
:100A9800F5007208840083137318831775088000A3
:100AA8005D2D770884008313781883170008F607EC
:100AB800F500750803190800F70AF20A7708840098
:100AC8008313781883170008F900720884008313C9
:100AD8007318831779088000F50B602D08007508D6
:100AE800F7007608F8007908FB007A08FC00F201A4
:100AF800F3017B08F5007C08F600F901FA012C25C2
:100B0800701C892DF501F60108001030F40003105F
:100B1800F70DF80DF20DF30D7B08F2027C08031CAB
:100B2800013EF30277140318A02D77107B08F20713
:100B38007C080318013EF307F40B8B2D7708F500AA
:100B48007808F6007208F0007308F10008008316B0
:100B580003178C130C14831203130800F001750893
:100B68007918F0070310F90C0310F50DF908031DA7
:100B7800B32D080072088400831373188317DA25CD
:100B8800F5008000F207D12D7208840083137318D2
:100B98008317DA25F500F607F207F50803190800A8
:100BA800DA25840A8000F50BD42D080078088A001D
:100BB8007708F70A0319F80A82000734203420342A
:100BC80045344A34503420342034073420344E34E9
:100BD8006F3472346D342E34203406345034723409
:100BE8006534613476342E340534533474346134C6
:100BF8007234743403343F343F343F340134203486
:100C0800BB013D08C80003190E2EEC202D08BB07B8
:0A0C1800C80B092E3B08D8000800A5
:02400E00D53F9C
:00000001FF
